:020000040000FA
:0400000006303A2864
:08000800A000030EA100831209
:100010008B1C32288B1031181428B11C3228643004
:10002000010203183128182800001628172818285C
:1000300019281A281B281C281D281E281F283110A3
:10004000B114A810031005190314AA0DA90DA80DC9
:10005000B00B322831152A08AF002908AE00280855
:10006000AD00B11081010B11210E8300A00E200EF6
:02007000090085
:0C007400203084008001840A6030040207
:10008000031C3C281230B000A3218316FF239000EC
:10009000831283160C308505870183128501870141
:1000A000073099000030831691009F008312C830FA
:1000B00083168100831231309000003083168C004B
:1000C000831210308B00831600309B001C141A081A
:1000D0008312BC00831610309B001C141A08831274
:1000E000BD00F42181018E018F010B118B100B10CB
:1000F0008C018B17892031199F20B30B872803109F
:1001000085190314B90DF03039020319182105229D
:100110007A286400311808000B1D08000B11B1107B
:1001200031141230B000051D9A28321483160113C1
:100130008312080032108316011783120800311150
:100140000130B7008B132030370783169B001C1437
:100150001A088312A400A500C030A5061030370786
:1001600083169B001C141A088312A3000030370763
:1001700083169B001C141A088312A2008B17321CD2
:10018000C72822090339A200A309A409A509220846
:100190002D02031D122923082E02031D12292408F3
:1001A0002F02031D122901303702031DDC283D18E0
:1001B000DC283D143E14AA2102303702031DE52835
:1001C000BD18E528BD143E14B12103303702031DCC
:1001D000EE283D19EE283D153E14B82104303702B3
:1001E000031DF728BD19F728BD153E14BF210530A2
:1001F0003702031D00293D1A00293D163E14C62171
:1002000006303702031D0929BD1A0929BD163E14FF
:10021000CD2107303702031D12293D1B12293D173E
:100220003E14D421B70A0830370203180800A22868
:100230000130B600B300B400B500B70085018701F6
:10024000B1138920B30B5629031085190314B90D76
:10025000F030390203197D29B40B562901303702D9
:100260000319DC21023037020319DF210330370282
:100270000319E221043037020319E5210530370262
:100280000319E821063037020319EB210730370242
:100290000319EE219630B4000330370232300319CF
:1002A000B4000430370232300319B400311D212963
:1002B0003111321C60292D090339AD00AE09AF0997
:1002C0002F1CB1132F1C2129B11B21292E182129E4
:1002D000B1178B1320303707BB002F08BA009021CD
:1002E00010303707BB002E08BA00902100303707C6
:1002F000BB002D08BA0090218B1785018701B70A32
:10030000B60108303702031C2129F42108003E1CE5
:1003100008003E101030BB003D08BA0090210800D4
:100320008B133A0883161C159A003B089B00553026
:100330009D00AA309D009C1464009C189C291C11EF
:1003400083128B170800FF30D000D415D515D615B1
:10035000D7150800BD103D11BD110230CE00D200EE
:1003600008003D103D11BD110130CE00D200080043
:100370003D10BD10BD118230CE00D20008003D10EE
:10038000BD103D114130CE00D2000800BD123D131A
:10039000BD130030CF00D30008003D123D13BD1344
:1003A0000230CF00D30008003D12BD12BD13013052
:1003B000CF00D30008000800013085060800023095
:1003C0008506080001308506080002308506080011
:1003D000303085060800103085060800203085067C
:1003E00008002230850608003D18AA21BD18B12159
:1003F0003D19B821BD19BF213D1AC621BD1ACD2115
:100400003D1BD421BD1BDB2108008F080319080008
:100410008F0196308E00D00FBF2AD00ABD1A372A1E
:10042000521C372A521F282AD41C192AD4015415C9
:10043000452A541D1E2AD401D415452AD41D232A29
:10044000D4015416452A541E452AD401D414452AF1
:10045000541D2D2AD4015416452AD41D322AD40104
:100460005416452A541E452AD401D414452AD41CB6
:100470003C2AD4015415452A541D412AD401D415CF
:10048000452A541E452AD4015415BD1A6E2AD21C81
:100490006E2AD21F5F2AD51C502AD50155157C2AF9
:1004A000551D552AD501D5157C2AD51D5A2AD501A9
:1004B00055167C2A551E7C2AD501D5147C2A551D3B
:1004C000642AD50155167C2AD51D692AD5015516F1
:1004D0007C2A551E7C2AD501D5147C2AD51C732A6A
:1004E000D50155157C2A551D782AD501D5157C2AAC
:1004F000551E7C2AD5015515531C8D2A561D832A5D
:10050000D60156169B2AD61D882AD60156169B2A36
:10051000561E9B2AD601D6149B2AD61C922AD60197
:1005200056159B2A561D972AD601D6159B2A561E6C
:100530009B2AD6015615D31CAC2A571DA22AD701D7
:100540005716BA2AD71DA72AD7015716BA2A571EF7
:10055000BA2AD701D714BA2AD71CB12AD7015715FE
:10056000BA2A571DB62AD701D715BA2A571EBA2A52
:10057000D701571587214E08D2004F08D3005008E5
:10058000D1000C305405031D85100C305505031D9A
:1005900005100C305605031D85120C305705031D40
:1005A000051251080E020318E92A12305405031DE2
:1005B000851412305505031D051412305605031D10
:1005C000851612305705031D0516FF30500203191A
:1005D00008008F08031D0800892051080E02031C23
:1005E000E92A18305405031D851006305405031DF3
:1005F000851418305505031D051006305505031DDB
:10060000051418305605031D851206305605031DC6
:10061000851618305705031D051206305705031DB2
:0406200005160800B3
:084000000E000300030008009C
:02400E00CC01E3
:10420000010003000300030003000200020002009B
:1042100002000000000000000000FF00FF00FF009F
:10422000000000000000000000000000000000008E
:104230000000C000C000C000C000FF00FF00FF0081
:104240000100C300F300CF00FF00C300F300CF0064
:10425000FF00C300F300CF00FF00FF00FF00FF00DE
:10426000FF00FF00FF00FF00FF00FF00FF00FF0056
:10427000FF00FF00FF00FF00FF00FF00FF00FF0046
:10428000FF00FF00FF00FF00FF00FF00FF00FF0036
:10429000FF00FF00FF00FF00FF00FF00FF00FF0026
:1042A000FF00FF00FF00FF00FF00FF00FF00FF0016
:1042B000FF00FF00FF00FF00FF00FF00FF00FF0006
:1042C000FF00FF00FF00FF00FF00FF00FF00FF00F6
:1042D000FF00FF00FF00FF00FF00FF00FF00FF00E6
:1042E000FF00FF00FF00FF00FF00FF00FF00FF00D6
:1042F000FF00FF00FF00FF00FF00FF00FF00AA001B
:00000001FF
